:020000020000FC
:1000000008C04AC118951895189530C118951895CB
:1000100018950FEFEEEFF3E0C895001609F001BE5A
:100020004427332755276627DD2410E02227EE24B6
:10003000662704E1902EA92CB92CC92C0FE001BD34
:1000400006E9802E0CE2502E06ED302E06E008BBAD
:1000500008E107BB01E005BFB199186000E00EBBE5
:10006000E09A0DB30F3FC1F0802E01E00EBBE09A85
:100070000DB30F3F89F0502E02E00EBBE09A0DB396
:100080000F3F51F00078102B03E00EBBE09A0DB348
:100090000F3F11F00074102B09E000BF782C00E432
:1000A0000BBF01E003BF32BE02E009BF789410FD30
:1000B00003C011FDC1C0FBCF072D761451F02AF00B
:1000C0000A95061531F07A9404C00395061509F0D7
:1000D0007394072D1E7F78143AF00819055082F1A9
:1000E00017FF08C017FD0EC0082D0719055042F173
:1000F00017FF08C012FF0EC0442716FF486016FD08
:10010000406108C012FF06C04427426016FF4061EC
:1001100016FD48600395402E13FD06C0442021F0D3
:1001200064EBB898C09A00C00695051532F0BA94F1
:1001300019F01B7F4427A92C0AC0A92CB92C07C091
:1001400013FFB89A44274424AA9409F4146013FFB7
:10015000AECF55FF08C0D394D7FEC098D7FCC09A45
:10016000B19B5F701AC054FF11C063FF08C05F707D
:10017000762F72957770751712F4C09A01C0C098E7
:100180005061B19B94CFDD24506291CF503029F45F
:10019000C09AB89AB19B51E18ACF513061F452E1D3
:1001A000D7FE85CF872C00E00EBB8DBAF894E29A7B
:1001B000E19A78947CCF523019F553E1D7FE77CF8E
:1001C0001B7F4427781422F01F77072D081903C0DE
:1001D0001068082D07190650502E01E00EBB5DBABD
:1001E000F894E29AE19A7894E199FECF02E00EBB8E
:1001F000012F00780DBBF894E29AE19A789457CFDA
:100200005330B9F454E1D7FE15C01B7F442703E0F7
:100210000EBB781417FD22F017FF12F41F7B01C0EC
:100220001064012F00740DBBF894E29AE19A78945F
:1002300001C03DCF177F3BCFA8951D7F639522302E
:1002400041F0CA9449F41B7F4427A92C2227EE24AD
:100250002ECF2227EE24C92C13FD29CF41FFB998B8
:1002600041FDB99A662309F4C09821CF32BE1FB66A
:10027000E39409F4239578943395341512F0C398D8
:10028000C498351539F43327C398C49843FDC39AED
:1002900044FDC49A1FBE18952FB6B29B04C02FBD53
:1002A00012602FBE18956FB411602FBE1895286389
:1002B000290930322F3230303462792E2E2E4861A7
:1002C0006E6E65532E2E2E2848616E6E65732E4C11
:0A02D000757840474D582E646529EB
:00000001FF
